:100000000C94B5040C94FC040C94FC040C94FC04B7
:100010000C94FC040C94FC040C94FC040C94FC0460
:100020000C94FC040C94FC040C94240E0C94F60E1A
:100030000C94FC040C94FC040C94FC040C94FC0440
:100040000C94FC040C941A230C94FC040C94FC04F3
:100050000C94FC040C94AC1C0C94FC040C94FC0458
:100060000C94FC040C94FC040C94FC040C94FC0410
:100070000C94FC040C94FC040C94FC040C94FC0400
:100080000C94FC040C94FC040C94FC040C94FC04F0
:100090000C94FC040C94FC040C94FC040C94FC04E0
:1000A0000C94FC040C94FC040C94FC04630F850F6A
:1000B0007810850F7810CA0FED0F78104210551088
:1000C0003F133F136E136E13B113EB13F815F815AE
:1000D0000414F815F914F914CC15F815F815E315EE
:1000E000751901620262016202620035002B00E1B3
:1000F00000E100E00000001E00140004001D0002EA
:10010000304E001F001A0016001B00E300E1002023
:1001100000080007000600AE002C002100150009B1
:1001200000190065744B00220017000A000500004A
:100130000029744C002A0000002800000008544CDC
:10014000002A00000028000000500023001C000BC3
:1001500000110000004F00240018000D001000E600
:1001600000520025000C000E0036002D002C002649
:100170000012000F0037004A00E50027001300338B
:100180000038002E00510030002F00347231724DC3
:1001900071000035002B00E100E100E00000001ECE
:1001A0000034000400330002304E001F00360012FD
:1001B000001400E300E1002000370008000D00AE4D
:1001C000002C002100130018000E0065744B002263
:1001D000001C000C001B00000029744C002A0000C9
:1001E000002800000008544C002A000000280000ED
:1001F000005000230009000700050000004F002404
:10020000000A000B001000E600520025000600174F
:10021000001A002F002C0026001500110019004ABA
:1002200000E50027000F0016001D00300051002ED1
:100230000038002D7231724D710000000000000086
:1002400000000000000000000000000000000000AE
:10025000000000000000000000000000000000009E
:10026000000000000000000000000000000000008E
:10027000000000000000000000000000000000007E
:1006200000000000000000000000000100010001C7
:10063000000100010000003A003F004400010001F9
:100640000001003B00400045000100010001003CAA
:1006500000410001000100010001003D00420001D5
:10066000000100010001003E004300010001000004
:100670000001000100010000000100000001000174
:1006800000010000005000000053003F0001005234
:100690000051000000390040004A004D004F0001A9
:1006A0000001002B005F005C005900620001005453
:1006B0000060005D005A0001300100550061005EDD
:1006C000005B0063000100560057005700580058B7
:1006D00071000001000100010001000100000001A3
:1006E0000001000100010001000100010001000102
:1006F000004C020100010001000100B200490101AB
:1007000000A80001000100B1004902010001000140
:10071000000100B500A800000001004900A9000088
:1007200000AA0000000100490001000000010000D3
:10073000000100B00001000100010000000100A55F
:10074000000100010001000100AC00A60001000151
:1007500000010001000100A70001000100010001EB
:1007600000010046000100010001000100AB00474C
:10077000004800010001000100000016034500725E
:100780000067006F0044006F007800200045005AA9
:1007900000000016034500720067006F0044006F00
:1007A000007800200045005A0000000403090409F5
:1007B000026D00040100A0FA090400000103010118
:1007C00000092111010001223F00070581030800F3
:1007D0000A090401000103010200092111010001BD
:1007E000224D000705820308000A090402000103E4
:1007F00000000009211101000122360007058303D2
:1008000008000A0904030001030000000921110186
:1008100000012239000705840310000112011001B4
:1008200000000008EDFE07130100010200010501B0
:100830000906A101050719E029E71500250195081A
:1008400075018102050819012905950575019102B7
:1008500095017503910105071900297715002501F8
:10086000957875018102C005010980A101850216F4
:10087000010026B7001A01002AB700751095018102
:1008800000C0050C0901A1018503160100269C0288
:100890001A01002A9C02751095018100C00501090A
:1008A00002A1010901A10005091901290515002569
:1008B0000195057501810295017503810105010905
:1008C0003009311581257F95027508810609381593
:1008D00081257F950175088106050C0A380215816E
:1008E000257F950175088106C0C005010906A10193
:1008F000050719E029E71500250195087501810212
:1009000095017508810105081901290595057501ED
:1009100091029501750391010507190029FF150042
:1009200025FF950675088100C0000000000000004A
:1009300000000000010204060A0F17202C3A4A5D4D
:1009400071879DB3C7DAE9F5FCFFFCF5E9DAC7B3B7
:100950009D87715D4A3A2C20170F0A060402010098
:100960000000000000000000000011241FBECFEFB7
:10097000DAE0DEBFCDBF04B603FE27C08091ED01F3
:100980009091EE01A091EF01B091F0018730904B72
:10099000A740B04BD1F41092ED011092EE011092ED
:1009A000EF011092F00114BE84B7877F84BF0FB6A9
:1009B000F894A895809160008861809360001092FF
:1009C00060000FBEE0E0FFE3099511E0A0E0B1E0B8
:1009D000E6EDF9E402C005900D92A433B107D9F712
:1009E00021E0A4E3B1E001C01D92AD3EB207E1F702
:1009F0000E946B0B0C94E9240C940000613049F0C8
:100A0000623059F488E00E94941A89E00E94941A96
:100A100004C0FC018281811103C080E090E0089550
:100A200080EE90E00895089556985E9825982D9848
:100A300026982E9827982F988091B1019091B20115
:100A4000A091B301B091B40190FF02C0259A2D9AF4
:100A50008091B5019091B601A091B701B091B80114
:100A60000297A105B10511F4269A2E9A0E94B110A1
:100A700081FF02C0279A2F9A08950C941405569866
:100A80005E9825982D9826982E9827982F988FEF66
:100A900090E0909389008093880090938B008093DE
:100AA0008A0090938D0080938C00259A2D9A2FEFC9
:100AB00080E792E0215080409040E1F700C00000C4
:100AC000269A2E9A2FEF80E792E0215080409040A6
:100AD000E1F700C00000279A2F9A2FEF80E792E0FD
:100AE000215080409040E1F700C0000025982D98EB
:100AF0002FEF80E792E0215080409040E1F700C066
:100B0000000026982E982FEF80E792E02150804039
:100B10009040E1F700C0000027982F9856985E9803
:100B200025982D9826982E9827982F98089589EA29
:100B30008093800089E08093810024982C983F98CE
:100B40008AB18F748AB96E98479A8BB1806B8BB9D2
:100B5000769A0E943F050C94130580E28093000171
:100B60008091340181110EC00E94FC0581E08093C8
:100B700034012FEF83ED90E3215080409040E1F766
:100B800000C0000080E40E940206809300018111F1
:100B90002EC00E942C0680930001811128C00E9463
:100BA0002C0680930001811122C08FE30E942C0645
:100BB0008093000181111BC00E94240680E40E94E2
:100BC000020680930001811112C08CE00E942C0665
:100BD0008093000181110BC00E942C0680930001BC
:100BE000811105C08FE30E942C06809300010E94B2
:100BF00024068091000108951092B9008AE0809344
:100C0000B800089594EA9093BC009091BC0097FFBF
:100C1000FCCF9091B900987F983021F0903111F07D
:100C200081E008958093BB0084E88093BC008091AC
:100C3000BC0087FFFCCF8091B900887F883111F01C
:100C4000803471F780E0089584E98093BC0080913E
:100C5000BC0084FDFCCF08958093BB0084E88093A2
:100C6000BC008091BC0087FFFCCF9091B900987FB9
:100C700081E0983209F480E0089584E88093BC0014
:100C80008091BC0087FFFCCF8091BB0008958091CC
:100C90000001811115C080E40E94020680930001CA
:100CA00081110CC082E10E942C0680930001811109
:100CB00005C08FEF0E942C06809300010E9424063D
:100CC00084B1807F84B985B1807F85B98AB1837F03
:100CD0008AB98BB1837F8BB93E98469808950E945C
:100CE000AD05809300010E94470680B38C7080BBE5
:100CF00081B3836F81BBE4E4F1E0A6E3B1E011923C
:100D00001D9281E0E235F807D1F70C9497059F9288
:100D1000AF92BF92CF92DF92EF92FF920F931F9309
:100D2000CF93DF9380910001882379F08091350182
:100D30008F5F80933501811108C00E94AD058093BB
:100D40000001811102C00E943F0586E3E82E81E088
:100D5000F82E8701C0E0D0E0BB24B39492E0A92E26
:100D6000CC24C394D12CC730D10500F5809100016B
:100D7000811164C080E40E94020680930001811109
:100D800012C082E10E942C068093000181110BC0E9
:100D9000C6010C2E01C0880F0A94EAF780950E94C4
:100DA0002C06809300010E94240648C0CA30A1F09E
:100DB00028F4C83059F0C93061F005C0CC3089F052
:100DC00070F0CD3089F0209A289810C0219A299887
:100DD0000DC0229A2A980AC0239A2B9807C0529ACB
:100DE00001C0539A5B9802C03E9A4698E0EAEA95A1
:100DF000F1F78FB181708B25799902C032E001C083
:100E000030E0832B7C9902C034E001C030E0832BBA
:100E10007D9902C028E001C020E0822B7E9902C0AB
:100E200090E101C090E0892B9FB19095991F99277F
:100E3000991F9295990F907E892B0FC08091000188
:100E400081114AC080E40E94020680930001882339
:100E500081F1912C0E942406892DD8019C9198172C
:100E600019F08C93A09201010E94470621960F5F12
:100E70001F4FCE30D10509F076CF80910101882334
:100E800069F1815080930101882339F0EFE9FFE097
:100E90003197F1F700C0000021C0E4E4F1E0D70190
:100EA0008D917D018193B4E4EB16B1E0FB06B9F7B7
:100EB00015C083E10E942C06809300018111C9CFE7
:100EC00081E40E940206809300018111C2CF0E943A
:100ED0003D06982E9094BECF80E0BFCF0E943D0586
:100EE00081E0DF91CF911F910F91FF90EF90DF9004
:100EF000CF90BF90AF909F900895E82FF0E0EC5B0B
:100F0000FE4F8081089508958B3B910580F4883AC7
:100F1000910548F5853A9105D8F48430910508F09B
:100F2000B2C0019709F06EC081E090E00895803E64
:100F3000910508F467C0883E910508F4A4C09C019F
:100F4000205F31092031310508F05CC090650895BB
:100F5000853A910509F459C0863A910509F058C0BF
:100F600082E890E40895883A910509F454C0893ADA
:100F7000910509F453C08A3A910509F452C08B3A9D
:100F8000910509F451C08C3A910509F450C08D3A8D
:100F9000910509F44FC0803B910509F44EC08E3A8B
:100FA000910509F44DC08F3A910509F44CC0813B7D
:100FB000910509F44BC0823B910509F44AC0833B7B
:100FC000910509F449C0843B910509F448C0853B6B
:100FD000910509F447C0863B910509F446C0873B5B
:100FE000910509F445C0883B910509F444C0893B4B
:100FF000910509F443C08A3B910509F442C080E0A1
:1010000094E4089580E090E0089581E890E40895E4
:1010100083E890E4089582EE94E4089589EE94E4E0
:1010200008958AEE94E4089585EB94E4089586EBA0
:1010300094E4089587EB94E408958CEC94E4089587
:101040008DEC94E4089583E895E408958AE895E4A6
:10105000089582E995E4089584E995E4089581E28C
:1010600096E4089583E296E4089584E296E4089570
:1010700085E296E4089586E296E4089587E296E490
:1010800008958AE296E40895089524E5829FC001B8
:101090001124FC0126E0729FE00DF11D1124E60FE2
:1010A000F11DEE0FFF1FE551FF4F859194910895BB
:1010B000880F991FFC01E559F0408591949108959E
:1010C000880F991FFC01E551FF4F85919491089578
:1010D00024E5829FC0011124FC0146E0749FE00DCD
:1010E000F11D1124E60FF11DEE0FFF1FE551FF4F1B
:1010F000859194919C013A9521154FE1340708F4AC
:1011000025C13F512115304120F49F700E94600895
:1011100008959C0130532115304118F49927906CA3
:101120000895811520E5920769F40E941A164FEF81
:1011300084E39CE0415080409040E1F700C0000013
:101140000C94D11C813020E5920731F48091CC01C0
:1011500081608093CC0108959C0130552115304168
:1011600008F05CC0292F33272F7033272130310539
:10117000E9F4AC0164E0440F551F6A95E1F7442798
:101180005370BC016370772702C0220F331F6A952A
:10119000E2F73C68242B352B73E0880F991F7A9572
:1011A000E1F780769927822B932B08952230310521
:1011B00029F4982F8827816F906A0895233031058C
:1011C000A1F4AC0133E0440F551F3A95E1F7407E9E
:1011D00057708370992721E030E002C0220F331F3F
:1011E0008A95E2F7C9019C6816C02430310531F5B3
:1011F000AC0123E0440F551F2A95E1F7407E57705C
:101200008370992721E030E002C0220F331F8A95B6
:10121000E2F7C9019A68842B952B08959C013057F9
:101220002115304118F49F70906208959C01305848
:101230002115304118F49F70906A0895803E910501
:10124000E0F4803C910558F58133910509F46FC0B5
:1012500048F48932910509F463C08A32910509F492
:101260006DC072C089339105E9F082389105D1F0E3
:101270008533910509F44DC067C0833E910581F126
:1012800038F4803E9105B9F0823E9105D9F05CC0FA
:10129000863E910561F1873E9105A1F155C00E94FE
:1012A000580808952091DE0120FD02C021FF4CC0A6
:1012B00080EE90E049C08091DE0180FFF9CF89E3A4
:1012C00090E042C08091DE0182FF0EC08091DE017D
:1012D00084FF03C080E090E037C083EE90E034C02C
:1012E0008091DE0182FFF2CF82EE90E02DC08091EE
:1012F000DE0183FF0BC08091DE0184FDEBCF87EE22
:1013000090E022C08091DE0183FFF5CF86EE90E071
:101310001BC08091DE0185FF07C089E290E014C008
:101320008091DE0185FFF9CF85E390E00DC08091CB
:10133000DE0186FF07C08AE290E006C08091DE01F0
:1013400086FFF9CF81E390E00E9484070895089515
:10135000809162010895CF93DF9300D01F92CDB7A3
:10136000DEB79C018091E401843019F593E0998304
:101370003B832A839093E9008FEF9091E80081509E
:1013800095FD06C095ED9A95F1F700008111F5CF16
:101390008091E80085FF0DC040E050E063E070E020
:1013A000CE0101960E94180C8091E8008E77809300
:1013B000E8000F900F900F90DF91CF910895CF9399
:1013C000DF9300D01F92CDB7DEB72091E401243027
:1013D00021F522E029839B838A8383E08093E900BF
:1013E0008FEF9091E800815095FD06C095ED9A959C
:1013F000F1F700008111F5CF8091E80085FF0DC065
:1014000040E050E063E070E0CE0101960E94180CCD
:101410008091E8008E778093E8000F900F900F90F6
:10142000DF91CF9108959C018091E4018430F9F41B
:1014300082E08093E9009FEF8091E800915085FD64
:1014400006C085ED8A95F1F700009111F5CF8091E6
:10145000E80085FF0CC040E050E065E070E0C901A5
:101460000E94180C8091E8008E778093E800089520
:10147000CF93DF93EC018091E401843009F046C002
:1014800090910C019923D9F090910D019923B9F015
:101490008093E9008FEF9091E800815095FD06C0A0
:1014A00095E19A95F1F700008111F5CF8091E80060
:1014B00085FF2CC040E050E060E170E017C081E0A3
:1014C0008093E9008FEF9091E800815095FD06C070
:1014D00095ED9A95F1F700008111F5CF8091E80024
:1014E00085FF14C040E050E068E070E0CE010E944B
:1014F000180C8091E8008E778093E80080E1FE016F
:10150000A2E5B1E001900D928A95E1F7DF91CF91CC
:1015100008958091E301811109C00E94A90D0E94E4
:10152000060E8091E20084608093E200089510929C
:10153000E301089508950C9407230E94671C0E94FC
:101540000D230E94B1100C94A70942E061EC81E0E8
:101550000E94220D42E061EC82E00E94220D42E0F6
:1015600061EC83E00E94220D42E161EC84E00C9486
:10157000220D8091E601833009F455C030F48130AA
:1015800071F0823009F48EC008958A3009F47AC06F
:101590008B3009F460C0893009F09CC020C0809174
:1015A000E501813A09F096C08091E800877F809339
:1015B000E8008091E9019091EA01892B21F460E132
:1015C00082E591E003C060E080E090E070E00E947E
:1015D000630C8091E8008B778093E80008958091F8
:1015E000E501813209F076C08091E9019091EA012C
:1015F000009719F0039709F06DC08091E800877F8C
:101600008093E8008091E80082FD05C08091E401AC
:101610008111F8CF5FC08091F100809362018091C9
:10162000E8008B7753C08091E501813A09F052C000
:101630008091E9019091EA01892B09F04BC08091DA
:10164000E800877F8093E8008091E80080FFFCCF6E
:1016500080910C0136C08091E5018132D9F58091ED
:10166000E9019091EA01892BA9F58091E800877F33
:101670008093E8000E94570D8091E70180930C0150
:101680000C941A168091E501813221F58091E800D1
:10169000877F8093E8000E94570D8091E801809336
:1016A000630108958091E501813AA1F48091E800F9
:1016B000877F8093E8008091E80080FFFCCF8091D5
:1016C00063018093F1008091E8008E778093E800B9
:1016D0000C94570D089584B7877F84BF0FB6F89494
:1016E000A8958091600088618093600010926000EE
:1016F0000FBE90E080E80FB6F8948093610090935D
:1017000061000FBE0E9400110E94A90D0E94060EEA
:101710008091E20084608093E20078940E949110AE
:101720000E94021182E091E00E94AC100E94F5221A
:101730008091E401853069F40E94291C8091E201C6
:101740008823B1F30E94531C882391F30E94020C5A
:10175000EFCF0E940811ECCF292F3327233031051A
:10176000C9F060F42130310581F02230310509F0F3
:1017700041C08DE690E02FEA37E040C021323105CC
:10178000E1F02232310531F135C082E190E02CE107
:1017900038E034C099278130910549F028F002974C
:1017A00049F5EBE7F7E005C0EBEAF7E002C0E3E953
:1017B000F7E0849190E09F0121C06430D8F4E62FD7
:1017C000F0E0EE0FFF1FEE5DFE4F2081318189E0DA
:1017D00090E014C0643070F470E0FB01EE0FFF1F66
:1017E000E65EFE4F20813181FB01EA5EFE4F808183
:1017F00090E004C080E090E020E030E0FA01318326
:101800002083089580E189BD82E189BD09B400FE8D
:10181000FDCF8091D8008F7D8093D8008091E0002B
:1018200082608093E0008091E00081FDFCCF08950C
:10183000CF92DF92EF92FF920F931F93CF93DF939C
:10184000EC018B016A010E94760D811133C0C11435
:10185000D10439F0F60180819181081B190BC80F62
:10186000D91FE12CF12C0115110519F18091E80027
:1018700085FD16C08091E8008E778093E800C11442
:10188000D10449F0F60180819181E80EF91EF182C0
:10189000E08285E00FC00E94760D882321F30AC004
:1018A00089918093F10001501109FFEFEF1AFF0AAF
:1018B000DACF80E0DF91CF911F910F91FF90EF90F1
:1018C000DF90CF9008952091EB013091EC01261725
:1018D000370748F06115710539F42091E8002E773B
:1018E0002093E80001C0B901FC0120E061157105F9
:1018F00079F18091E4018823F1F18530F1F1809153
:10190000E80083FD3CC08091E80082FD2EC08091FC
:10191000E80080FFEBCF2091F3008091F20090E08F
:10192000922B6115710551F08830910538F42191A1
:101930002093F100615071090196F3CF21E00897DF
:1019400009F020E08091E8008E778093E800CECF08
:101950002111CFCF0AC08091E401882361F0853046
:1019600061F08091E80083FD0AC08091E80082FF69
:10197000F2CF80E0089582E0089583E0089581E049
:1019800008952091EB013091EC012617370748F0BC
:101990006115710539F42091E8002E772093E80055
:1019A00001C0B901FC0120E06115710591F1809140
:1019B000E401882309F440C0853009F43FC08091D8
:1019C000E80083FD3DC08091E80082FD2FC080913A
:1019D000E80080FFE9CF2091F3008091F20090E0D1
:1019E000922B6115710559F08830910540F42491CE
:1019F0002093F1003196615071090196F2CF21E0F8
:101A0000089709F020E08091E8008E778093E80045
:101A1000CBCF2111CCCF0AC08091E401882361F0A3
:101A2000853061F08091E80083FD0AC08091E80074
:101A300082FFF2CF80E0089582E0089583E0089568
:101A400081E00895982F973068F59093E9009817F2
:101A500039F07091EC002091ED005091F00003C03E
:101A6000242F762F50E021FD02C09F5FECCF3091F4
:101A7000EB003E7F3093EB003091ED003D7F3093E3
:101A8000ED003091EB0031603093EB007093EC008F
:101A90002093ED005093F0002091EE0027FDE5CF5C
:101AA00080E008958F708093E90081E0089580912F
:101AB000E50187FF11C08091E80082FD05C080919B
:101AC000E4018111F8CF11C08091E8008B770BC041
:101AD0008091E401882349F08091E80080FFF8CFED
:101AE0008091E8008E778093E80008952091E400CB
:101AF0003091E50095E64091EC00842F817040FF25
:101B000023C08091E80080FD1DC08091E4018823FE
:101B100099F0853099F08091EB0085FD11C04091DE
:101B2000E4005091E5002417350729F3915011F096
:101B30009A01E1CF84E0089582E0089583E008955A
:101B400081E0089580E008954091E80042FFDDCFF4
:101B500008950E94170E0E941F0EE0EEF0E08081B3
:101B600081608083E8EDF0E080818F77808319BC0D
:101B7000A7EDB0E08C918E7F8C9380818F7E8083E7
:101B80001092E30108950F931F93CF93DF930E9468
:101B9000170E0E941F0EC8EDD0E088818F778883D2
:101BA00088818068888388818F7D888319BC1092A2
:101BB000E4011092E0011092E2011092E10100EEC6
:101BC00010E0F80180818B7F808388818160888329
:101BD00042E060E080E00E94220DE1EEF0E08081D2
:101BE0008E7F8083E2EEF0E080818160808380815F
:101BF00088608083F80180818E7F80838881806106
:101C00008883DF91CF911F910F910895E8EDF0E067
:101C100080818F7E8083E7EDF0E08081816080832A
:101C200084E082BF81E08093E3010C94C30DE8ED72
:101C3000F0E080818E7F80831092E2000895109200
:101C4000DA001092E10008951F920F920FB60F92E2
:101C500011242F933F934F935F936F937F938F93B1
:101C60009F93AF93BF93EF93FF938091E10082FF27
:101C70000BC08091E20082FF07C08091E1008B7F62
:101C80008093E1000E9490108091DA0080FF1FC0D5
:101C90008091D80080FF1BC08091DA008E7F8093F6
:101CA000DA008091D90080FF0DC080E189BD82E11A
:101CB00089BD09B400FEFDCF81E08093E4010E945C
:101CC000890A05C019BC1092E4010E94970A80910C
:101CD000E10080FF19C08091E20080FF15C0809173
:101CE000E2008E7F8093E2008091E2008061809329
:101CF000E2008091D80080628093D80019BC85E012
:101D00008093E4010E949B0A8091E10084FF30C02F
:101D10008091E20084FF2CC080E189BD82E189BD11
:101D200009B400FEFDCF8091D8008F7D8093D8004C
:101D30008091E1008F7E8093E1008091E2008F7EB0
:101D40008093E2008091E20081608093E2008091C4
:101D5000E001882311F084E007C08091E30087FD53
:101D600002C081E001C083E08093E4010E949D0AEB
:101D70008091E10083FF29C08091E20083FF25C0AC
:101D80008091E100877F8093E10082E08093E4010D
:101D90001092E0018091E1008E7F8093E1008091BC
:101DA000E2008E7F8093E2008091E2008061809368
:101DB000E20042E060E080E00E94220D8091F000AD
:101DC00088608093F0000E949A0AFF91EF91BF9182
:101DD000AF919F918F917F916F915F914F913F91C3
:101DE0002F910F900FBE0F901F9018951F920F927A
:101DF0000FB60F9211242F933F934F935F936F93DE
:101E00007F938F939F93AF93BF93CF93DF93EF9382
:101E1000FF93C091E900CF708091EC00D82FD17072
:101E200080FDD0E81092E9008091F000877F8093D8
:101E3000F00078940E943A0F1092E9008091F0002F
:101E400088608093F000CD2BCF70C093E900FF91A4
:101E5000EF91DF91CF91BF91AF919F918F917F9142
:101E60006F915F914F913F912F910F900FBE0F9007
:101E70001F9018951F93CF93DF93CDB7DEB7AA9726
:101E80000FB6F894DEBF0FBECDBFE5EEF1E0809156
:101E9000F100819321E0ED3EF207C9F70E94B90AF3
:101EA0008091E80083FF24C18091E5019091E601D3
:101EB000492F50E04A30510508F01AC1FA01EA5A98
:101EC000FF4F0C949E24803881F0823809F010C1B5
:101ED0008091E9018F708093E9008091EB0085FB90
:101EE000882780F91092E90006C08091E101909165
:101EF000E201911182609091E800977F9093E80051
:101F00008093F1001092F100C8C0282F2D7F09F0B6
:101F1000EFC0882319F0823061F0EAC08091E701B8
:101F2000813009F0E5C0933009F080E08093E20150
:101F30002BC08091E701811127C08091E9018F704A
:101F400009F4D6C08093E9002091EB0020FF1CC06B
:101F5000933021F48091EB00806214C09091EB00EB
:101F600090619093EB0021E030E0A90102C0440FA2
:101F7000551F8A95E2F74093EA001092EA0080919B
:101F8000EB0088608093EB001092E9008091E800FC
:101F9000877F86C08111ACC01091E7011F778091C7
:101FA000E3008078812B8093E3008091E800877FB5
:101FB0008093E8000E94570D8091E80080FFFCCFDD
:101FC0008091E30080688093E300111102C082E0F9
:101FD00001C083E08093E4018BC08058823008F018
:101FE00087C08091E7019091E8018C3D53E095070F
:101FF00079F583E08A838AE289834FB7F894DE011A
:10200000139620E03EE051E2E32FF0E050935700BA
:10201000E49120FF03C0E295EF703F5FEF708E2FD9
:1020200090E0EA3010F0C79601C0C0968D939D9362
:102030002F5F243149F74FBF8091E800877F80935D
:10204000E8006AE270E0CE0101960E94630C14C0C1
:10205000AE014F5F5F4F6091E9010E94AC0BBC0184
:10206000892B09F445C09091E800977F9093E80090
:1020700089819A810E94C10C8091E8008B778093BE
:10208000E80036C08038A1F58091E800877F809312
:10209000E8008091E0018093F1008091E8008E7764
:1020A0008093E8000E94570D23C0811121C08091C8
:1020B000E7019091E80199270297D4F48091E80014
:1020C000877F8093E8008091E7018093E0010E9480
:1020D000570D8091E001811106C08091E30087FDDA
:1020E00002C081E001C084E08093E4010E94A50A5F
:1020F0008091E80083FF0AC08091E800877F809389
:10210000E8008091EB0080628093EB00AA960FB606
:10211000F894DEBF0FBECDBFDF91CF911F91089520
:102120000895CF938091E4018823A1F0C091E90044
:10213000CF709091EC00892F817090FD80E8C82BC2
:102140001092E9008091E80083FD0E943A0FCF7061
:10215000C093E900CF91089590936901809368013D
:102160000895E0916801F0916901309721F00190A4
:10217000F081E02D099480E00895E0916801F091EC
:102180006901309721F00280F381E02D09940895D0
:10219000E0916801F0916901309721F00480F581A8
:1021A000E02D099408952091660130916701281768
:1021B000390771F09093670180936601E09168019F
:1021C000F0916901309721F00680F781E02D0994A4
:1021D000089520916401309165012817390771F045
:1021E0009093650180936401E0916801F091690129
:1021F000309721F00084F185E02D09940895089529
:102200000C94FF100E946D1C0E946F060C94331DED
:10221000CF92DF92EF92FF920F931F93CF93DF93B2
:10222000CDB7DEB72B970FB6F894DEBF0FBECDBF8C
:102230000E9487068BE6C82E81E0D82E00E010E0D1
:10224000E02E802F0E947D07F60141916F01F82E4C
:10225000F426B1F40F5F1F4F0E30110589F78FEF91
:1022600089838A831B820E94761C8160782F9D83DC
:102270008C8349815A816B818D810E94AB1140C052
:102280009091CC0191FF04C08B870E9483078B85BE
:1022900020E030E04F2D50E0922FBA01022E02C014
:1022A000759567950A94E2F760FF24C02E83EF824C
:1022B00021E030E0690102C0CC0CDD1C9A95E2F708
:1022C00090E08C219D21892B09F420E028870E9431
:1022D000761C8160782F9A8789874E815F81688517
:1022E0008A850E94AB11F801E559FE4F8081C8260E
:1022F000C08206C02F5F3F4F2630310569F6AACF56
:102300000E941A200E94B11090916A018917A1F0D1
:102310000E94B11080936A012B960FB6F894DEBF2D
:102320000FBECDBFDF91CF911F910F91FF90EF9026
:10233000DF90CF900C94A7092B960FB6F894DEBFD0
:102340000FBECDBFDF91CF911F910F91FF90EF9006
:10235000DF90CF900895CF93DF93CDB7DEB72B9763
:102360000FB6F894DEBF0FBECDBF4F835887698785
:102370007A878B87DE01119686E0FD0111928A959E
:10238000E9F785E0FE01379601900D928A95E1F715
:1023900049815A816B817C818D819E810E94AE181A
:1023A0002B960FB6F894DEBF0FBECDBFDF91CF9155
:1023B0000895CF93C82F882309F4C1C0823859F4F7
:1023C0000E94B11081FDBBC089E30E944B1B0E949B
:1023D000031C89E30CC0833879F40E94B11080FD9E
:1023E000AEC083E50E944B1B0E94031C83E50E9444
:1023F0008A1BCF910C94031C843859F40E94B110AD
:1024000082FD9DC087E40E944B1B0E94031C87E451
:10241000EECF8CEF8C0F813A48F48C2F0E945A2219
:1024200081118DC08C2F0E944B1BE3CF80E28C0F5B
:10243000883048F4C77081E001C0880FCA95EAF778
:102440000E94CC1BD6CF8BE58C0F833078F4C53A35
:1024500029F0C63A31F083E890E005C081E890E0C9
:1024600002C082E890E0CF910C94D31088E58C0FE5
:10247000833108F064C0C83A39F1C93A41F1CA3A27
:1024800049F1CB3A51F1CC3A59F1CD3A61F1C03B27
:1024900069F1CE3A71F1CF3A79F1C13B81F1C23B9A
:1024A00089F1C33B91F1C43B99F1C53BA1F1C63B16
:1024B000A9F1C73BB1F1C83BB9F1C93BC1F1CA3B76
:1024C000C9F180E090E038C082EE90E035C089EE3E
:1024D00090E032C08AEE90E02FC085EB90E02CC0F7
:1024E00086EB90E029C087EB90E026C08CEC90E072
:1024F00023C08DEC90E020C083E891E01DC08AE805
:1025000091E01AC082E991E017C084E991E014C01B
:1025100081E292E011C083E292E00EC084E292E098
:102520000BC085E292E008C086E292E005C087E237
:1025300092E002C08AE292E0CF910C94E910CF9130
:102540000895882309F44BC0823859F40E94B110D1
:1025500081FF45C089E30E944B1B0E94031C89E355
:102560000CC0833871F40E94B11080FF38C083E53D
:102570000E944B1B0E94031C83E50E948A1B0C9443
:10258000031C843859F40E94B11082FF28C087E4EC
:102590000E944B1B0E94031C87E4EFCF9CEF980F17
:1025A000913A58F390E2980F983050F4877091E088
:1025B00001C0990F8A95EAF7892F0E94D21BDFCFBD
:1025C0009BE5980F933020F480E090E00C94D310BA
:1025D000885A833120F480E090E00C94E91008954B
:1025E000882321F00E94CC1B0C94031C089588239F
:1025F00021F00E94D21B0C94031C0895BF92CF922D
:10260000DF92EF92FF920F931F93CF93DF9300D04F
:1026100000D000D0CDB7DEB77C0185E0F701DE0148
:10262000119601900D928A95E1F7F70183819481CB
:10263000892B09F4DDC2908181818F3F19F49F3F7E
:1026400009F4D6C2F7010281258122952F70998362
:102650008A8389819A812E830E940A1B182FB92EA2
:102660000E94091B0E94D019EB2DE295EF704E2FAE
:1026700050E0FA01E05AFF4F2E810C949E248B2DDE
:10268000807F9B2D9F70F92E882319F0F29480EFA4
:10269000F822002349F0FF2009F457C28F2D0E9431
:1026A000DC1B0E94031C51C2812F0E94A112FF203B
:1026B00009F49EC28F2D0E94E21B26960FB6F89455
:1026C000DEBF0FBECDBFDF91CF911F910F91FF9065
:1026D000EF90DF90CF90BF900C94031C3B2D307F88
:1026E0008B2D8F70303211F08295807F112319F07D
:1026F000113021F12CC00023B9F0222309F490C13C
:10270000213009F08DC126960FB6F894DEBF0FBEBA
:10271000CDBFDF91CF911F910F91FF90EF90DF9090
:10272000CF90BF900C94EC1B222319F0213009F4B8
:102730005FC28E830E94EF1B8E8186C1002321F031
:10274000223008F055C26CC1211152C27DC1002354
:1027500021F0222309F464C1F8C1222309F474C1D1
:1027600009C28B2D86958695837019F08130D1F042
:102770003FC2002321F0812F9B2D937002C080E087
:1027800090E026960FB6F894DEBF0FBECDBFDF9166
:10279000CF911F910F91FF90EF90DF90CF90BF905E
:1027A0000C94D310002321F0812F9B2D937002C035
:1027B00080E090E026960FB6F894DEBF0FBECDBF46
:1027C000DF91CF911F910F91FF90EF90DF90CF900D
:1027D000BF900C94E910812F002319F00E94221F52
:1027E00002C00E948A1F26960FB6F894DEBF0FBE65
:1027F000CDBFDF91CF911F910F91FF90EF90DF90B0
:10280000CF90BF900C940F208B2D837009F075C072
:102810000111EEC1812F829586958770880F880FF0
:10282000912F9F70C92ED12CE12CF12C082E04C0C1
:10283000CC0CDD1CEE1CFF1C0A94D2F714FF12C056
:102840000FE010E020E030E004C0000F111F221F55
:10285000331F8A95D2F7C901B801609570958095AC
:10286000909503C060E070E0CB014B2D46954695F6
:1028700043704230C1F060F56C297D298E299F2973
:10288000413051F126960FB6F894DEBF0FBECDBF92
:10289000DF91CF911F910F91FF90EF90DF90CF903C
:1028A000BF900C94F7196C297D298E299F292696B3
:1028B0000FB6F894DEBF0FBECDBFDF91CF911F9151
:1028C0000F91FF90EF90DF90CF90BF900C94131A70
:1028D0000E94F719C701B60126960FB6F894DEBF1D
:1028E0000FBECDBFDF91CF911F910F91FF90EF9061
:1028F000DF90CF90BF900C94DB19002319F08B2D43
:10290000817001C08695882309F472C1812F829558
:1029100086958770880F880F912F9F70C92ED12CB4
:10292000E12CF12C082E04C0CC0CDD1CEE1CFF1C8D
:102930000A94D2F714FF12C00FE010E020E030E05C
:1029400004C0000F111F221F331F8A95D2F7C9013F
:10295000B801609570958095909503C060E070E037
:10296000CB014B2D4695469543704230C1F060F542
:102970006C297D298E299F29413051F126960FB669
:10298000F894DEBF0FBECDBFDF91CF911F910F91A5
:10299000FF90EF90DF90CF90BF900C94D11A6C29EC
:1029A0007D298E299F2926960FB6F894DEBF0FBE8B
:1029B000CDBFDF91CF911F910F91FF90EF90DF90EE
:1029C000CF90BF900C94ED1A0E94D11AC701B601A6
:1029D00026960FB6F894DEBF0FBECDBFDF91CF9124
:1029E0001F910F91FF90EF90DF90CF90BF900C94CC
:1029F000B51A103FD1F118F4103E50F4A1C0123FA7
:102A000009F463C008F44CC0133F09F473C098C0C4
:102A10001F708B2D8F710023A1F00E944E1A812F01
:102A200026960FB6F894DEBF0FBECDBFDF91CF91D3
:102A30001F910F91FF90EF90DF90CF90BF900C947B
:102A4000F0120E946F1A812F26960FB6F894DEBFFF
:102A50000FBECDBFDF91CF911F910F91FF90EF90EF
:102A6000DF90CF90BF900C94F7120023A9F02111B2
:102A7000BFC08B2D8F7126960FB6F894DEBF0FBEA8
:102A8000CDBFDF91CF911F910F91FF90EF90DF901D
:102A9000CF90BF900C94941A223008F0A9C0E9CFCF
:102AA0000023A9F08B2D8F7126960FB6F894DEBF08
:102AB0000FBECDBFDF91CF911F910F91FF90EF908F
:102AC000DF90CF90BF900C944E1A002359F38B2DBA
:102AD0008F7126960FB6F894DEBF0FBECDBFDF9183
:102AE000CF911F910F91FF90EF90DF90CF90BF900B
:102AF0000C946F1A002399F08B2D8F7126960FB6C8
:102B0000F894DEBF0FBECDBFDF91CF911F910F9123
:102B1000FF90EF90DF90CF90BF900C94391A2696DB
:102B20000FB6F894DEBF0FBECDBFDF91CF911F91DE
:102B30000F91FF90EF90DF90CF90BF900C942F1AE1
:102B40000023A9F0222309F4ADCF812F26960FB6DA
:102B5000F894DEBF0FBECDBFDF91CF911F910F91D3
:102B6000FF90EF90DF90CF90BF900C94D91122236B
:102B700009F4ADCF812F26960FB6F894DEBF0FBEB5
:102B8000CDBFDF91CF911F910F91FF90EF90DF901C
:102B9000CF90BF900C94A1124B2D4F70612FC701A5
:102BA0000E94FE0426960FB6F894DEBF0FBECDBF7E
:102BB000DF91CF911F910F91FF90EF90DF90CF9019
:102BC000BF900C9453194B2D4F70612FC70126965F
:102BD0000FB6F894DEBF0FBECDBFDF91CF911F912E
:102BE0000F91FF90EF90DF90CF90BF900C9444082E
:102BF00026960FB6F894DEBF0FBECDBFDF91CF9102
:102C00001F910F91FF90EF90DF90CF90BF900895AC
:102C10000E94E91B0E94BE1B0E94031C0E94BF2051
:102C20000E940F2080E090E00E94D31080E090E0AE
:102C30000C94E9100E94D91B0C9408160E940A1BE0
:102C4000292F22952F702C3030F42A3048F422504E
:102C5000223078F405C02C3041F02F3031F009C01B
:102C6000803E48F0803F29F406C093FB882780F916
:102C7000089580E0089581E00895CF93DF9300D018
:102C800000D01F92CDB7DEB70F900F900F900F902E
:102C90000F90DF91CF910895CF93DF9300D000D0B4
:102CA00000D0CDB7DEB726960FB6F894DEBF0FBEC4
:102CB000CDBFDF91CF9108951F93CF93DF93C09144
:102CC000790116E080917A01C81799F0D0E01C9F35
:102CD000F0011D9FF00D1124E558FE4F40815181F8
:102CE00062817381848195810E944C162196C77000
:102CF000E9CFDF91CF911F9108954091AB015091A1
:102D0000AC016091AD017091AE018091AF019091E5
:102D1000B0010C944C168091B00182958F7009F02F
:102D200054C08091AD01882309F44FC0809179018E
:102D3000A0917A014091AE015091AF016091AB0139
:102D40007091AC01B6E08A1709F43FC090E04115DC
:102D50005105C1F17F3F11F46F3FA1F1B89FF00120
:102D6000B99FF00D1124E558FE4F218127132AC089
:102D70002081261327C02281211124C02381348180
:102D80002417350710F421503109241B350B283C3A
:102D90003105C0F42091B0012F7020612093B00163
:102DA00026E0289FF001299FF00D1124E058FE4FE6
:102DB00080818F70806180838BEA91E00E94FE1297
:102DC0000C945C1601968770BECF0895CF92DF9267
:102DD000EF92FF920F931F93CF93DF93CDB7DEB7A0
:102DE00062970FB6F894DEBF0FBECDBF8C0185E0B1
:102DF000F801DE011D9601900D928A95E1F7D80148
:102E00004C9111965C91119712966C918091AE0144
:102E10009091AF01009709F475C13091AB017091A9
:102E2000AC017F3F19F43F3F09F46CC1F801C38046
:102E3000D480E090AD01EE2009F4BEC02091B00135
:102E4000C816D90628F0D601A81BB90BCD0104C0BD
:102E5000809590958C0D9D1DFF24F394883C9105E1
:102E600078F0F12C207F09F0C4C07C2DD98AC88A63
:102E700089890E943D168BEA91E00E94FE12AFC044
:102E8000822F807F09F045C0571313C0431311C030
:102E900061110FC02F7020612093B0010E947D1638
:102EA0008BEA91E00E94FE128091B001F8018583C7
:102EB0002EC0CD2819F15F3F11F44F3FF9F0F62EE7
:102EC00061111CC08091790120917A0136E082174E
:102ED00009F45BC090E0389FF001399FF00D112498
:102EE000E558FE4F7181571306C07081471303C028
:102EF0007281711103C001968770E9CFF62E6623A7
:102F000009F41CC18091B00181608093B001F12C63
:102F100015C1571309C0431307C0611105C0809143
:102F2000B001F8018583C8C04D875E878D859E8579
:102F30006A8B0E941E166A898823D1F16623C1F12B
:102F40002091B001822F82958F7090E0029774F0EB
:102F50008091AB019091AC0198878F831986DB86B5
:102F6000CA862C87CE0107960E94FE1286E0F801E1
:102F7000ABEAB1E001900D928A95E1F70E948B16C1
:102F80000E947D16FF24F394D9C04D875E878D85FE
:102F90009E850E940A1B292F22952F70223008F04F
:102FA000C1C09F7009F0BBC0805E883008F4C6C005
:102FB000C8010E94FE12E6CFC816D90608F453C015
:102FC000F601E81BF90BCF01883C910508F450C0CD
:102FD000F12C7C2DD98AC88A89890E943D16EBEA9A
:102FE000F1E086E0DF011D928A95E9F70E947D16E7
:102FF000A5C0571314C0431312C0611110C08091B3
:10300000B001F8018583C8010E94FE1286E0EBEA58
:10301000F1E0DF011D928A95E9F7FE2C8FC04D8704
:103020005E878D859E856A8B0E941E166A8988231D
:1030300009F4BECF662309F4BBCF2091B001822FE3
:1030400082958F7090E002970CF490CF8091AB0145
:103050009091AC019A8389831B82DD82CC822E837E
:10306000CE01019681CF809590958C0D9D1DACCFA2
:10307000F62E662309F49CCF571333C0431331C097
:103080002091B00120FD24C0822F82958F70482F9F
:1030900050E041155105E1F0D80115962C93159794
:1030A0004F30510549F08F5F982F9295907F822F76
:1030B0008F70892B15968C93C8010E94FE1286E0B2
:1030C000F801ABEAB1E001900D928A95E1F78ECF5D
:1030D00086E0F801ABEAB1E001900D928A95E1F744
:1030E0002DC04D875E878D859E850E941E1681119D
:1030F0003DCF8091B00181608093B001C8010E94F2
:10310000FE121CC0662309F453CF4D875E878D8560
:103110009E850E941E16882309F44ACF27CF81116D
:1031200043CF0CC0243008F043CF9F7009F43CCF4C
:10313000D80115969C91907F09F036CF8F2D62961D
:103140000FB6F894DEBF0FBECDBFDF91CF911F91B8
:103150000F91FF90EF90DF90CF9008951F93CF9342
:10316000DF93CDB7DEB72C970FB6F894DEBF0FBE56
:10317000CDBF4F83588769877A878B879C87CE011D
:1031800007960E94E616882371F08A859B85892B15
:1031900009F441C088858F3F09F065C08F818F3F5A
:1031A00009F061C038C086E0FE013796DE01119655
:1031B00001900D928A95E1F76A857B85611571050D
:1031C00051F1FF81E885EF3F11F4FF3F21F120919C
:1031D0007A0130E0C9010196877099274091790101
:1031E00050E08417950709F447C0F983EA837D838B
:1031F0006C8396E0929FD001939FB00D1124A55847
:10320000BE4FFE01319601900D929A95E1F78093A1
:103210007A010E945C1616E08091790190917A0102
:103220008917B9F1189FC001112485589E4F0E943B
:10323000E616882371F1E09179011E9FF0011124B7
:10324000E558FE4F4081518162817381848195816F
:103250000E944C168091790190E001968770992721
:1032600080937901D9CF4F81588569857A858B857F
:103270009C850E944C16CFCF0E941A1610927A019C
:1032800010927901EBEAF1E086E0DF011D928A9568
:10329000E9F72C960FB6F894DEBF0FBECDBFDF91D5
:1032A000CF911F910895EF92FF920F931F93CF93A9
:1032B000DF938C01892B09F46CC0F12CEE24E3948C
:1032C000E8012196F8018491843740F4843008F0B5
:1032D00051C0813081F0823019F15BC0853709F42B
:1032E00044C0A8F19CE7980F903708F052C08F7740
:1032F0000E94A11241C00E5F1F4FFE01849190E217
:10330000980F983050F48770FE2D01C0FF0F8A95FA
:10331000EAF78F2F0E94DC1B14C00E94D9112DC028
:103320000E5F1F4FFE01849190E2980F983060F479
:103330008770FE2D01C0FF0F8A95EAF78F2F0E943C
:10334000E21B0E94031C19C00E94A11216C00E5F4E
:103350001F4FFE01C491CC2381F08FE99FE00197BC
:10336000F1F700C00000C150F6CF0E5F1F4FFE0105
:10337000F49003C00E94D9118E018F2D882309F487
:103380009FCFEFE9FFE03197F1F700C000008150D7
:10339000F5CFDF91CF911F910F91FF90EF9008959E
:1033A00008956093B5017093B6018093B70190932F
:1033B000B8010C9408160F931F930091B50110915A
:1033C000B6012091B7013091B801DC01CB01802B0F
:1033D000912BA22BB32B8093B5019093B601A093B0
:1033E000B701B093B8011F910F910C9408160F9379
:1033F0001F930091B5011091B6012091B701309152
:10340000B801DC01CB0180239123A223B323809355
:10341000B5019093B601A093B701B093B8011F9185
:103420000F910C9408160F931F930091B501109102
:10343000B6012091B7013091B801DC01CB018027A2
:103440009127A227B3278093B5019093B601A0934B
:10345000B701B093B8011F910F910C940816109208
:10346000B1011092B2011092B3011092B4010C9408
:10347000081641E050E060E070E004C0440F551FC2
:10348000661F771F8A95D2F74093B1015093B2011E
:103490006093B3017093B4010C94081641E050E0BE
:1034A00060E070E004C0440F551F661F771F8A95C7
:1034B000D2F78091B1019091B201A091B301B09186
:1034C000B401482B592B6A2B7B2B4093B1015093AD
:1034D000B2016093B3017093B4010C94081641E0FB
:1034E00050E060E070E004C0440F551F661F771F76
:1034F0008A95D2F740955095609570958091B1016D
:103500009091B201A091B301B091B4014823592325
:103510006A237B234093B1015093B2016093B301BE
:103520007093B4010C94081641E050E060E070E044
:1035300004C0440F551F661F771F8A95D2F78091EC
:10354000B1019091B201A091B301B091B4014827AB
:1035500059276A277B274093B1015093B2016093AA
:10356000B3017093B4010C9408160F931F9300914C
:10357000B1011091B2012091B3013091B401DC018D
:10358000CB01802B912BA22BB32B8093B101909375
:10359000B201A093B301B093B4011F910F910C94A9
:1035A00008160F931F930091B1011091B201209161
:1035B000B3013091B401DC01CB0180239123A2231C
:1035C000B3238093B1019093B201A093B301B09360
:1035D000B4011F910F910C9408160F931F93009143
:1035E000B1011091B2012091B3013091B401DC011D
:1035F000CB0180279127A227B3278093B101909315
:10360000B201A093B301B093B4011F910F910C9438
:1036100008160895CF92DF92EF92FF920F931F93B7
:10362000CF93DF938C01C090B101D090B201E090B4
:10363000B301F090B4018091B5019091B601A091D1
:10364000B701B091B801C82AD92AEA2AFB2ACFE1EA
:10365000D0E0D701C6010C2E04C0B695A79597956A
:1036600087950A94D2F780FF07C0B8018C2F0E947B
:1036700068088130910531F4219758F7B80180E04E
:103680000E946808DF91CF911F910F91FF90EF90FA
:10369000DF90CF90089590910C019923F1F09091D3
:1036A0000D019923D1F0982F9695969596959F3078
:1036B00080F5E0910E01F0910F01E90FF11D877087
:1036C00021E030E0A90102C0440F551F8A95E2F7BE
:1036D000CA019181892B8183089520910E01309137
:1036E0000F01F90132969FEF40E05191851789F063
:1036F0009F3F19F4511101C0942F4F5F4E30A9F72D
:103700009F3F39F0F901E90FF11D97FDFA9582838A
:103710000895089590910C019923F9F090910D016D
:103720009923D9F0982F9695969596959F3028F5E0
:10373000E0910E01F0910F01E90FF11D877021E07A
:1037400030E0A90102C0440F551F8A95E2F7CA0173
:103750008095918189238183089520910E01309174
:103760000F01F9013296205F3F4F9081891301C00C
:1037700010823196E217F307C1F7089581E090E0D7
:10378000E0910E01F0910F01E80FF91F10820196F0
:1037900080319105A9F708959091CB01892B8093F1
:1037A000CB01089580959091CB0189238093CB0123
:1037B00008951092CB0108959091CA01892B8093AE
:1037C000CA01089580959091CA0189238093CA0106
:1037D00008951092CA0108958093B9010895109236
:1037E000B901089580910E0190910F01FC0131966D
:1037F0009C01205F3F4F80E0919191118F5FE21714
:10380000F307D1F70895E0910E01F0910F01809137
:10381000CB018083E0910E01F0910F0190818091A6
:10382000CA01892B80838091B901882361F0E091DE
:103830000E01F0910F019081892B80830E94F21B71
:1038400081111092B90180910E0190910F010C9499
:10385000BD108091E401843011F120E488E190E012
:103860000FB6F894A895809360000FBE2093600077
:1038700083B7817F846083BF83B7816083BF78947F
:10388000889583B78E7F83BF0FB6F894A8958091F3
:103890006000886180936000109260000FBE089500
:1038A00008950C94501CCF930E94511C0E948706CF
:1038B0000E94501CC0E08C2F0E947D07811104C023
:1038C000CF5FCE30C1F701C081E0CF9108950E9453
:1038D0001A160E94B1100C94A70982E084BD93E0EF
:1038E00095BD9AEF97BD80936E0008952FB7F89419
:1038F0008091CD019091CE01A091CF01B091D001E6
:103900002FBF0895CF92DF92EF92FF920F931F93F4
:103910002FB7F8944091CD015091CE016091CF0125
:103920007091D0012FBF6A017B01EE24FF248C012E
:1039300020E030E0C016D106E206F30610F4415054
:1039400051099A01281B390BC9011F910F91FF9052
:10395000EF90DF90CF9008951F920F920FB60F92C5
:1039600011248F939F93AF93BF938091CD0190913A
:10397000CE01A091CF01B091D0010196A11DB11D42
:103980008093CD019093CE01A093CF01B093D0014D
:10399000BF91AF919F918F910F900FBE0F901F908D
:1039A00018950E94A90DF8942FEF87EA91E621500F
:1039B00080409040E1F700C0000087E090EBDC0120
:1039C0008093ED019093EE01A093EF01B093F0018D
:1039D0009CE088E10FB6F894A895809360000FBE34
:1039E00090936000FFCFEF92FF920F931F93CF93BE
:1039F000DF93D82FC0E08C2F0E947D0700E010E0FD
:103A0000E82EF12CC701002E02C0959587950A94E7
:103A1000E2F780FD06C00F5F1F4F0630110591F7DA
:103A200009C0602F7C2F80E00E9445088D13F3CFE2
:103A300081E004C0CF5FCE30F1F680E0DF91CF911E
:103A40001F910F91FF90EF900895CF93C82F8CE2B4
:103A50000E94F31C882321F08C2FCF910C94F31C2F
:103A600080E0CF910895CF930E947A1E811102C009
:103A70000E94601EC5E6C15049F00E9487068FE390
:103A80009CE90197F1F700C00000F5CF89E20E94A0
:103A9000251D811113C18AE20E94251D81110E94FA
:103AA000601E85E00E94251D81110E94D11C0E948C
:103AB000851E8093CC0187E00E94251D8823A9F1F3
:103AC0008BE10E94251D882351F08091CC0181FB60
:103AD000222720F991E0922790FB81F90EC08EE019
:103AE0000E94251D882361F08091CC0182FB222752
:103AF00020F991E0922790FB82F98093CC0115C0C8
:103B000080E10E94251D9091CC01882341F093FB18
:103B1000222720F981E0822780FB93F904C0892FB6
:103B2000809580FB90F99093CC018091CC010E940C
:103B3000891E0E94971E8093DE0180EE0E94251D43
:103B4000882341F08091DE01982F909590FB80F9B9
:103B50008093DE0189E30E94251D882359F080911E
:103B6000DE0181FB222720F991E0922790FB81F969
:103B70008093DE0182EE0E94251D882359F08091FA
:103B8000DE0182FB222720F991E0922790FB82F947
:103B90008093DE0186EE0E94251D882359F08091D6
:103BA000DE0183FB222720F991E0922790FB83F925
:103BB0008093DE0183EE0E94251D882359F08091B9
:103BC000DE0184FB222720F991E0922790FB84F903
:103BD0008093DE0185E30E94251D882359F08091A2
:103BE000DE0185FB222720F991E0922790FB85F9E1
:103BF0008093DE0181E30E94251D882359F0809186
:103C0000DE0186FB222720F991E0922790FB86F9BE
:103C10008093DE0181E10E94251D882359F0809167
:103C2000DE0187FB222720F991E0922790FB87F99C
:103C30008093DE018091DE010E949B1E8091DE0157
:103C400087FB882780F980930D0187E20E94251D5C
:103C5000C82F8EE10E94251D8111C2608FE10E9454
:103C6000251D8111C46080E20E94251D8111C8605C
:103C700081E20E94251D8111C06182E20E94251D02
:103C80008111C06283E20E94251D8111C06484E21B
:103C90000E94251D882311F0C06802C0CC2329F0A2
:103CA0008C2F0E94921E6C2F03C00E948E1E682FC4
:103CB00070E080E090E0CF910C94D119CF910895FD
:103CC0006DEE7EEF80E090E00E94D42460E082E020
:103CD00090E00E94C62460E083E090E00E94C62449
:103CE00060E084E090E00E94C62460E085E090E01F
:103CF0000C94C62480E090E00E94C02421E08D3E18
:103D00009E4F09F020E0822F089582E090E00C940D
:103D1000B824682F82E090E00C94C62483E090E001
:103D20000C94B824682F83E090E00C94C62484E0BF
:103D300090E00C94B824682F84E090E00C94C624A2
:103D40008091D30180FF0BC06091130185E0689FD3
:103D5000B001112475956795759567952BC081FF06
:103D600009C06091130185E0689FB0011124759529
:103D7000679520C082FF07C06091130185E0689FAE
:103D8000B001112417C09091D4019923D1F0609112
:103D90001201961788F72091130185E0289F900162
:103DA0001124929FA001939F500D112470E0CA012D
:103DB0000E948A246038710540F46115710519F478
:103DC00006C065E070E0862F08958FE7089581E0D2
:103DD00008958091D30180FF08C06091110170E0C7
:103DE000759567957595679521C081FF06C06091AF
:103DF000110170E07595679519C082FF04C060914C
:103E0000110170E010C09091D401992399F0609154
:103E100010019617A0F780911101899FC00111240C
:103E200070E00E948A246038710540F461157105C4
:103E300019F406C061E070E0862F08958FE70895B9
:103E400081E00895803F21F40E94A01E819504C066
:103E5000813F29F40E94A01E8093D7010895823FDC
:103E600021F40E94A01E819504C0833F29F40E9482
:103E7000A01E8093D6010895893F19F40E94E91E7F
:103E800005C08A3F31F40E94E91E81958093D801D4
:103E900008958B3F21F40E94E91E819504C08C3F58
:103EA00029F40E94E91E8093D9010895843F21F4EA
:103EB0008091D501816017C0853F21F48091D501A3
:103EC000826011C0863F21F48091D50184600BC0CF
:103ED000873F21F48091D501886005C0883F31F487
:103EE0008091D50180618093D50108958D3F21F4A3
:103EF0008091D30181600BC08E3F21F48091D3016A
:103F0000826005C08F3F29F48091D3018460809343
:103F1000D3010895803F39F48091D70187FF6CC0A9
:103F20001092D70169C0813F29F48091D7011816FA
:103F3000BCF362C09091D601823F29F497FF5CC028
:103F40001092D60159C0833F19F41916CCF354C00E
:103F5000893F41F48091D80118160CF04DC01092A1
:103F6000D8014AC08A3F29F48091D80187FF44C014
:103F7000F6CF8B3F39F48091D90187FF3DC0109275
:103F8000D9013AC08C3F29F48091D9011816BCF3AD
:103F900033C0843F21F48091D5018E7F17C0853FC7
:103FA00021F48091D5018D7F11C0863F21F480914D
:103FB000D5018B7F0BC0873F21F48091D501877F8E
:103FC00005C0883F31F48091D5018F7E8093D50163
:103FD00013C08D3F21F48091D3018E7F0BC08E3FA3
:103FE00021F48091D3018D7F05C08F3F29F480910A
:103FF000D3018B7F8093D3018091D60181110EC0B4
:104000008091D70181110AC08091D801811106C029
:104010008091D901811102C01092D401089585EDDB
:1040200091E00E94C8100E94761C9093D201809368
:10403000D10108951F93CF93DF938091D101909187
:10404000D2010E94821CAC019091D401992321F0ED
:104050002091140130E006C0209115018AE0289FCC
:10406000900111244217530708F485C08091D601AE
:10407000C091D701D091D8011091D901811107C009
:10408000C11175C0D11173C0111171C074C09F3FAF
:1040900019F09F5F9093D401181624F40E94A01E7B
:1040A0008093D6018091D60187FF05C00E94A01E93
:1040B00081958093D6011C1624F40E94A01E809343
:1040C000D7018091D70187FF05C00E94A01E81956E
:1040D0008093D7016091D601662331F1C091D70159
:1040E000CC2311F1062E000C770B880B990B0E9444
:1040F000912323E333E343E35FE30E94F5230E942C
:1041000059236093D6016C2FCC0F770B880B990B3A
:104110000E94912323E333E343E35FE30E94F5230B
:104120000E9459236093D7011D1624F40E94E91EB2
:104130008093D8018091D80187FF05C00E94E91EB5
:1041400081958093D801111624F40E94E91E809372
:10415000D9018091D90187FF05C00E94E91E819590
:104160008093D901DF91CF911F910C940F209F3F35
:1041700009F08FCFA0CFDF91CF911F910895E5ED8A
:10418000F1E085E0DF011D928A95E9F71092D401F4
:104190001092D3010895833081F128F4813059F0D1
:1041A0008230D1F00895853009F449C0B8F18630E5
:1041B00009F456C0089580911501262F30E0280F8C
:1041C000311D2F3F310524F4680F609315010895C8
:1041D0008FEF80931501089580911401262F30E010
:1041E000280F311D2F3F310524F4680F609314010F
:1041F00008958FEF80931401089580911301262F65
:1042000030E0280F311D2F3F310524F4680F6093F3
:10421000130108958FEF8093130108958091120187
:10422000262F30E0280F311D2F3F310524F4680F71
:104230006093120108958FEF809312010895809189
:104240001101262F30E0280F311D2F3F310524F4B6
:10425000680F6093110108958FEF80931101089505
:1042600080911001262F30E0280F311D2F3F31059E
:1042700024F4680F6093100108958FEF809310016C
:104280000895833011F128F4813049F0823091F0A3
:104290000895853081F120F18630C1F10895809133
:1042A0001501681720F4861B80931501089510925C
:1042B0001501089580911401681720F4861B8093DE
:1042C0001401089510921401089580911301681744
:1042D00020F4861B80931301089510921301089512
:1042E00080911201681720F4861B809312010895B3
:1042F00010921201089580911101681720F4861B15
:104300008093110108951092110108958091100178
:10431000681720F4861B80931001089510921001F5
:1043200008950F931F938D3109F46BC008F03FC0BF
:104330008E3009F47DC0C0F4873009F46EC068F493
:10434000863009F0AFC08091CC01817F8E7F809351
:10435000CC0181E08093DB01A6C0883009F458C00D
:104360008B3009F49BC09EC0863109F497C078F465
:10437000803109F470C0813109F094C00E941A168E
:1043800090910D0181E0892780930D0187C08931CB
:1043900009F484C08B3109F085C08091CC0181FB88
:1043A000222720F991E0922790FB81F94AC08533BA
:1043B00009F45BC048F4873209F457C008F45AC0C6
:1043C000893209F452C06EC0833438F48A3308F05D
:1043D00067C0883309F462C065C0833409F445C0FE
:1043E000883409F05FC00E941A160FEF13ED20E326
:1043F000015010402040E1F700C000000E94D11C95
:104400004DC00E9413230E94B1100E94A70946C00C
:104410000E94851E0E94971E41C09091CC01892F59
:10442000817090FF12C0917F9E7F9093CC013BC022
:104430008091CC0182FB222720F991E0922790FB0A
:1044400082F98093CC01992349F18091CC0181605C
:104450008093CC0123C08091CC0183FB222720F9DB
:1044600091E0922790FB83F9ECCF61E070E080E06F
:1044700090E010C08D5141E050E060E070E08A01B2
:104480009B0104C0000F111F221F331F8A95D2F712
:10449000C901B8010E94D1190E941A1681E003C017
:1044A0008953E9CF80E01F910F91089580E008952E
:1044B0000C945622CF93C82F8091DB01813079F084
:1044C00018F08230E9F187C0E0910E01F0910F0100
:1044D0008081813169F0823209F07FC009C0E091AA
:1044E0000E01F0910F018081813111F0823261F46F
:1044F0008C2F0E945822811104C08C2F0E94912180
:104500001DC081E090E01AC08C2F0E9456228111BC
:1045100014C0C43179F048F4CB3079F0C03109F0DF
:1045200060C082E08093DB0108C0C93219F0C83353
:1045300021F057C01092DB0154C081E0817053C05C
:10454000C93289F118F5C43171F1A8F4C73009F006
:1045500046C08AE08093150194E19093140193E0A2
:10456000909313018093120188E08093110188E2F7
:104570008093100134C0CE51C63088F5EC2FF0E0A6
:10458000E65DFE4F80818093DA0129C0CE34E9F0E8
:1045900020F4CB3421F56AE013C0C13579F0C2357F
:1045A000F1F461E00DC08091DA01882319F01092D6
:1045B000DA0115C081E08093DB0115C061E006C01F
:1045C0008091DA010E94CB200AC06AE08091DA0172
:1045D0000E94412104C01092DB0180E004C081E010
:1045E00002C080E0ABCFCF910895E1E8F0E0808198
:1045F000886080838081816080838FB7F89493E0A6
:104600009093890090ED909388008FBF0895EFE616
:10461000F0E08081826080830895EFE6F0E08081A1
:104620008D7F80830895EFE6F0E0908182E0892716
:10463000808308951F920F920FB60F9211242F932B
:104640003F934F935F936F937F938F939F93AF931A
:10465000BF93EF93FF938091DC019091DD01019670
:104660009093DD018093DC01811103C082E00E9400
:10467000A709E091DD01E695E695F0E0E75DF64FEC
:10468000E4918091DC018E1303C080E00E94A709B1
:10469000FF91EF91BF91AF919F918F917F916F911A
:1046A0005F914F913F912F910F900FBE0F901F90F0
:1046B00018950E9460236894B1110C94EF2308951B
:1046C0000E94D42388F09F5798F0B92F9927B751AB
:1046D000B0F0E1F0660F771F881F991F1AF0BA95A6
:1046E000C9F714C0B13091F00E94EE23B1E00895F3
:1046F0000C94EE23672F782F8827B85F39F0B93FE5
:10470000CCF3869577956795B395D9F73EF4909558
:104710008095709561957F4F8F4F9F4F0895E894D6
:1047200009C097FB3EF490958095709561957F4FF9
:104730008F4F9F4F9923A9F0F92F96E9BB279395A7
:10474000F695879577956795B795F111F8CFFAF4B7
:10475000BB0F11F460FF1BC06F5F7F4F8F4F9F4FE8
:1047600016C0882311F096E911C0772321F09EE846
:10477000872F762F05C0662371F096E8862F70E0AC
:1047800060E02AF09A95660F771F881FDAF7880F86
:104790009695879597F9089557FD9058440F551FA2
:1047A00059F05F3F71F04795880F97FB991F61F0B3
:1047B0009F3F79F087950895121613061406551F2A
:1047C000F2CF4695F1DF08C0161617061806991F96
:1047D000F1CF86957105610508940895E894BB278B
:1047E00066277727CB0197F908950E9408240C9437
:1047F00079240E946B2438F00E94722420F09523C3
:1048000011F00C9462240C94682411240C94EF236E
:104810000E94CC2370F3959FC1F3950F50E0551F74
:10482000629FF001729FBB27F00DB11D639FAA2705
:10483000F00DB11DAA1F649F6627B00DA11D661F54
:10484000829F2227B00DA11D621F739FB00DA11D75
:10485000621F839FA00D611D221F749F3327A00D2F
:10486000611D231F849F600D211D822F762F6A2FCB
:1048700011249F5750409AF0F1F088234AF0EE0F30
:10488000FF1FBB1F661F771F881F91505040A9F75D
:104890009E3F510580F00C9462240C94EF235F3FFF
:1048A000E4F3983ED4F3869577956795B795F79599
:1048B000E7959F5FC1F7FE2B880F911D9695879511
:1048C00097F9089597F99F6780E870E060E0089590
:1048D0009FEF80EC089500240A9416161706180618
:1048E0000906089500240A941216130614060506F4
:1048F0000895092E0394000C11F4882352F0BB0F85
:1049000040F4BF2B11F460FF04C06F5F7F4F8F4FE7
:104910009F4F089597FB072E16F4009407D077FD5C
:1049200009D00E94A42407FC05D03EF490958195FF
:104930009F4F0895709561957F4F0895EE0FFF1F6B
:104940000590F491E02D0994AA1BBB1B51E107C00F
:10495000AA1FBB1FA617B70710F0A61BB70B881F0F
:10496000991F5A95A9F780959095BC01CD0108959E
:10497000F999FECF92BD81BDF89A992780B5089527
:10498000A8E1B0E042E050E00C94DB24262FF99936
:10499000FECF1FBA92BD81BD20BD0FB6F894FA9A22
:1049A000F99A0FBE019608950E94C624272F0C94F1
:1049B000C724DC01CB01FC01F999FECF06C0F2BD92
:1049C000E1BDF89A319600B40D9241505040B8F7CD
:0649D0000895F894FFCFEA
:1049D6002002A809380A130ADF09AB090101BA0146
:1049E60028080A03140A3F4D3639EA089D08670865
:1049F6002E08C107DA07F3070C08010203040506AF
:044A06000708090094
:00000001FF
